:1000000008308A000B2A0000FF00030E8301A100C4
:100010000A08A0008A010408A2007708A300780853
:10002000A4007908A5007A08A6007B08A70083131E
:1000300083120B1E1D288B1842288C308400801ED2
:1000400023288C1A45288C308400001C29280C1881
:1000500048288C308400801C2F288C184B282208BC
:1000600084002308F7002408F8002508F900260872
:10007000FA002708FB0020088A00210E8300FF0EEB
:100080007F0E09008A110A129A298A110A12802801
:100090008A110A1268298A110A1278290A108A100C
:1000A0000A11820730342E34353400340A108A1095
:1000B0000A1182075734443454340D340A3400345E
:1000C0000A108A100A11820743344F344D344D34DC
:1000D00041344E34443420344534523452344F3455
:1000E00052340D340A34003464008C1E742818080D
:1000F000EE001A08F800EE1C7F28181218160034BB
:10010000A0307107840083130317EA010408E90093
:100110006A10831B6A140313742003176908840090
:1001200083136A18831778088000A0307107840051
:1001300083130008243C031DA6280130F200F101BE
:10014000243083160313A00083120317F208031947
:1001500063297108043C031DC52804307102703EF8
:10016000F800FA010318FA0A7808E8007A08E900AA
:10017000A0307107840083130008EA006808840037
:100180008313691883176A0880000130F10771082A
:10019000063C03186329F201F10101300313EF005B
:1001A000831621082F3C0318D9282108393C03184D
:1001B000E9282108403C0318E1282108463C03189F
:1001C000E9282108603C031816292108663C031C15
:1001D000162922082F3C0318F1282208393C03185D
:1001E00001292208403C0318F9282208463C03183C
:1001F00001292208603C031816292208663C031CCA
:1002000016292208393C031807290930A2070F30A4
:10021000A2052108393C03180F290930A1070F3026
:10022000A1050310210D2204F30019298312EC16F5
:10023000831625082F3C031821292508393C03186B
:1002400031292508403C031829292508463C031874
:1002500031292508603C03185E292508663C031CEB
:100260005E2926082F3C031839292608393C031833
:1002700049292608403C031841292608463C031812
:1002800049292608603C03185E292608663C031CA1
:100290005E292608393C03184F290930A6070F307C
:1002A000A6052508393C031857290930A5070F3042
:1002B000A5050310250D2604F400612983126C178F
:1002C00083168312031703138C128A110A122F2824
:1002D000D80B74290130D0070318D10A0319D20AA8
:1002E0000319D30A0F30D8000C108A110A122F28D4
:1002F000D90B84290130D4070318D50A0319D60A6B
:100300000319D70A6230D9008C108A110A122F28DB
:1003100083160C1083125308DD005208DC005108CC
:10032000DB005008DA0058080F3CE20083160C147A
:10033000831200346C1CA729EC18A7296C1AA72972
:1003400088210616831606128312EC14AC296C1849
:10035000AC296C19AC296C158B108A110A122F2844
:100360008C1EB4297420B02983168612831286123B
:100370000034F51575088316870000308312871D39
:100380000130F700770D8316C900C90DC90DF8308B
:10039000C90575157508870000308312071D0130E7
:1003A000F700F70DF70DFC30F705770883164904C1
:1003B000CB00F5147508870000308312871C0130CC
:1003C000F7000310F70D770883164B04CD00751462
:1003D0007508870000308312071C013083164D0416
:1003E0008312ED00B021EF0183168C16C03083120A
:1003F0008B048A150A128C2A7C08840083137D18CA
:10040000831703173A088000840A8001FC0A031945
:10041000FD0A031300340317B91B202A0F30F7001D
:10042000380EF7050A3077020318192A3030F7071B
:100430001B2A3908F7077708BA000313FC210317B2
:100440000F30B8050A3038020318282A30302A2A1B
:10045000B9133908B8073808BA000313FC2100346F
:1004600003173908BE003808BD003E08FA003D08F1
:10047000840083137A18831780080319432ABD0A5E
:100480000319BE0A352A3B08FA003A088400831390
:100490007A18831780080319672A3C08003C031860
:1004A000672A3A08840083133B1883170008C100A9
:1004B0003D08840083133E18831741088000BD0A5D
:1004C0000319BE0ABA0A0319BB0ABC03432A3D0832
:1004D000840083133E18831780013808F800390818
:1004E000F900031300348316861283128616003433
:1004F00073220317BA01B9013A08013C031CA02A70
:10050000031D862A3908903C031CA02AF51775089C
:100510008316031387008312871B932A0317BA01DC
:10052000B901992A031364001030F700F70B962ADB
:100530000317B808031D6400B90A0319BA0A7C2A14
:100540000313B02100340C1EA32A03174108031320
:1005500099008A110A12E22A4030840083170008A9
:100560000319C32A0130F800BF30F7006400F70B0D
:10057000B62AF80BB42A4A30F700F70BBD2A000060
:100580006400800BB22A003403173F100313732258
:100590000317BC013C08043C031CFC2A03136E1324
:1005A0000317BD0139083D020318E82A3B08FA0089
:1005B0003A08840083133B1883170008C000C10069
:1005C0000313A32A0317BA0A0319BB0ABD0AD22AC6
:1005D00003136E1BF42A4F080317C0000313AC2249
:1005E00003173F14FC2A03134F080317C00003131B
:1005F000AC220317BC0ACA2A0313B0210030031728
:100600003F180130F800031300340130FD001030B2
:10061000FC003F300317BA000313FC216D080317D9
:10062000B8005730B90003130B2220300317BA006B
:100630000313FC2101300317B9001030B8008316F2
:100640000313490883120317BB00831603134808DA
:1006500083120317BA001030BC000313302279084C
:100660008316C9007808C800CA014A0848078400F0
:1006700083134918831780080319402BCA0A352BA6
:1006800083120317B801031378226D080317B8000B
:10069000831603134A0883120317B9008316031342
:1006A000490883120317BB008316031348088312FB
:1006B0000317BA000313C422F808031D652B0A3080
:1006C0000317C0000313AC22452B00348316C9085E
:1006D0000319722B8312EF080319702B8316722BE8
:1006E000662B83168312EF08031D7A2B0030F80067
:1006F0008A2B8A2B6D087302031D852BEC1A852B20
:10070000EF010130F8008A2B8A2BEC12EF01003048
:10071000F8008A2B8A150A12FA2A83164908FA0069
:100720004808840083137A1883170008CC004B080C
:10073000FA004A08840083137A18831700084C02D1
:10074000031DB92B4908FA004808840083137A185E
:1007500083178008031DAF2B0030F800D22B490807
:10076000FA004808C80A0319C90ACA0A0319CB0AB9
:100770008E2B4908FA004808840083134918831710
:100780000008CC004B08FA004A08840083134B1879
:10079000831700084C020318D02BFF30FA00D12B2E
:1007A0000130F8008312003483160C108312D30139
:1007B000D201D101D0010F30D80083160C148C1057
:1007C0008312D701D601D501D4016230D900831636
:1007D0008C148312061583160611831207127512E4
:1007E00075088316870083128716F512750883161D
:1007F000870083126C148A150A120E2B2030831680
:10080000D400D001D101D201D3014B08FA004A082B
:10081000F9004908F8004808F7000310771C1E2C5F
:100820004C08D0074D0803184D0FD1074E08031888
:100830004E0FD2074F0803184F0FD307D30CD20C1B
:10084000D10CD00CFA0CF90CF80CF70CD40B0D2CC5
:10085000831200348E30F70083164D08F8004C08E0
:10086000F900FA01F808031D3F2C7908F800F90196
:100870000830F702F808031D3F2CF701472C03103E
:10088000F81B462CF90DF80DF7033F2CF8138312D3
:10089000003483164C080319BA2CD40050080319ED
:1008A000BA2CD40703185B2C7F30D402031CBA2C5B
:1008B0000319BA2C5F2C8130D4070318BA2C5408C2
:1008C000F700F801F901FA014D08D800D8174E08D1
:1008D000D7004F08D6001830D400D501561C882CFC
:1008E0005308FA07031C7A2CF90A031D7A2CF80A1C
:1008F0000319D5175208F907031C812CF80A0319AC
:10090000D5175108CE00CE174E08F8070318D51793
:10091000D50DF80CF90CFA0CD80CD70CD60C03102A
:10092000D40B6D2C0130F7070318BA2CF81B9F2C41
:10093000D80DFA0DF90DF80DF7030319BA2CD81FCD
:10094000B02CFA0A031DB02CF90A031DB02CF80ACA
:10095000031DB02CF80CF90CFA0CF70A0319BA2C89
:100960004D08D5005108D506D51FB82CF817BE2C58
:10097000F813BE2CF701F801F901FA0183120034D3
:10098000B630F700FA01F901F80183165008510456
:1009900052045304031DCE2CF701DB2C0310F81B6B
:1009A000DA2CD00DD10DD20DD30DFA0DF90DF80DB5
:1009B000F70BCE2CF813831200348030831CE32C09
:1009C0008316D50683128316DA01DB015108D9009C
:1009D0005508D90650080319D12DD800F70054083E
:1009E0000319DA2DD8020319762D031C342D55086E
:1009F000DE00DE175608DD005708DC00DB010310BF
:100A0000DE0CDD0CDC0CDB0CD80BFE2CD91F0B2D07
:100A10005A14EE2D5A1058105A16D33084008313EE
:100A2000032E5A12D91B1E2D581C292DDE0CDD0C4D
:100A3000DC0CDB0CF70A0319E92D292DDE1B2C2D0C
:100A40000310DB0DDC0DDD0DDE0DF7030319E92DC1
:100A50001E2D5A17962D5A135108D900D91F322D21
:100A6000DE17E22DDE13E22D5408D800F7005008FF
:100A7000D8025108DE00DE175208DD005308DC0002
:100A8000DB010310DE0CDD0CDC0CDB0CD80B402D85
:100A9000D91F4D2DDA14EE2DDA105810DA16D73092
:100AA00084008313032EDA12D91B602D581C6B2D82
:100AB000DE0CDD0CDC0CDB0CF70A0319E92D6B2DC9
:100AC000DE1B6E2D0310DB0DDC0DDD0DDE0DF703DF
:100AD0000319E92D602DDA17962DDA135508D90080
:100AE000D91F742DDE17E22DDE13E22D5508DE002E
:100AF000DE175608DD005708DC00D91F832DDE13F2
:100B00005A15EE2D5A11DB015810D330840083138F
:100B1000032ED91BAC2D5108D900581C962DDE0C84
:100B2000DD0CDC0CDB0CF70A0319E92DDB1FA72D0C
:100B3000DC0A031DA72DDD0A031DA72DDE0A031DF8
:100B4000A72DDE0CDD0CDC0CF70A0319E92D5A1B6E
:100B50002B2DDA1B6D2DCB2D8030DE06DE1FB42D44
:100B6000EE2D5508D900C12D5108D900DE08031D0E
:100B7000C12DDD08031DC12DDC08031DC12DF701AA
:100B8000E22DDE1BCB2D0310DB0DDC0DDD0DDE0DAC
:100B9000F70BC12DE92DD91FCF2DDE17E22DDE1366
:100BA000E22D5408F7005508DE005608DD0057080E
:100BB000DC00E22D5008F7005108DE005208DD008D
:100BC0005308DC005E08F8005D08F9005C08FA00D4
:100BD000212EF701F801F901FA01212EDB01DC09D0
:100BE000DD09DE09DB09DB0A031DFC2DDC0A031D20
:100BF000FC2DDD0A0319DE0A5A180A2DDA184C2DCD
:100C00005A19822DB12D0008DC07031C0D2EDD0AB8
:100C1000031D0D2EDE0A0319581484030008DD0796
:100C2000031C152EDE0A0319581484030008801FC4
:100C3000803ADE07031858145A1A112DDA1A532D68
:100C4000892D8312003483165008B63CD000FA0177
:100C50005108D400D1170310D10CD20CD30CFA0CCC
:100C6000F90CF80CF70CD00B2B2ED41F422EF709E1
:100C7000F809F909FA09F70A0319F80A0319F90A30
:100C80000319FA0A83120034F701F801F901FA0195
:100C90008316DC01DD01DE01DF015B085A04590423
:100CA00058040319832E2030E0000310D40DD50D15
:100CB000D60DD70DDC0DDD0DDE0DDF0D5B085F02FF
:100CC000031D6C2E5A085E02031D6C2E59085D022E
:100CD000031D6C2E58085C02031C7D2E5808DC0294
:100CE0005908031C590FDD025A08031C5A0FDE0273
:100CF0005B08031C5B0FDF020314F70DF80DF90D01
:100D0000FA0DE00B552EDC3084008313831200347F
:100D100004088316CC00CB1F9A2ECC03CC16C8092E
:100D2000C909CA09CB09C80A0319C90A0319CA0A99
:100D30000319CB0A3B30D3009A30D200CA30D1001D
:100D4000D0010A30CE004B08D7004A08D600490827
:100D5000D5004808D4005308DB005208DA005108D7
:100D6000D9005008D8008312442600088316C80012
:100D7000840A0008C900840A0008CA00840A00081E
:100D8000CB00F708031DD72E4E08013A0319D72EC2
:100D90004C080319D92E0F394E020319D12E03180E
:100DA000012FCC1B012F4C1BD92E2030F92E2030C7
:100DB000CC05CC1EE82ECC127708CC002D30831247
:100DC0000317BA000313FC2183164C08F700CC016B
:100DD0003030CC1EF92ECC127708CC002D30831287
:100DE0000317BA000313FC2183164C08F700CC014B
:100DF0003030F707770883120317BA000313FC217A
:100E000083165308D7005208D6005108D500500861
:100E1000D400DB01DA01D9010A30D800831244265C
:100E20007A088316D3007908D2007808D1007708B1
:100E3000D000CE0BA32E83120034861483168610A6
:100E40000130FD001030FC002A3083120317BA0075
:100E50000313FC216D080317B8005730B9000313C2
:100E60000B2201300317B9001030B80083160313AA
:100E7000490883120317BB00831603134808831223
:100E80000317BA001030BC00031330227908831610
:100E9000C9007808C800CA014A08480784008313BB
:100EA0004918831780080319572FCA0A4C2F831239
:100EB0000317B801031378226D080317B8008316CF
:100EC00003134A0883120317B90083160313490852
:100ED00083120317BB0083160313480883120317FA
:100EE000BA000313C422F808031D7C2F0A3003172D
:100EF000C0000313AC225C2F861083168610831269
:100F0000003400306C180130F700770D8316C900EB
:100F1000C90DC90DF830C90500308312EC1B013032
:100F2000F700F70DF70DFC30F70577088316490435
:100F3000CB0000308312EC180130F7000310F70DDE
:100F4000770883164B04CD00003083126C190130F2
:100F500083164D04F600FD013B30FC007608831239
:100F60000317B8005730B90003130B220D300317D5
:100F7000BA000313FC210A300317BA000313FC2143
:100F80008316C9013B30C80083121D278A150A1237
:100F9000302BFD013B30FC008316C801480883124A
:100FA0004E2000380319DE2F8316C80A8312031758
:100FB000BA000313FC218316CE2F83120D300317C2
:100FC000BA000313FC210A300317BA000313FC21F3
:100FD0008316C9013B30C80083121D278A150A12E7
:0A0FE000422BF12F8A150A12642B30
:101000006C1C8428EC1C84285D088316CB0083129A
:101010005C088316CA0083125B088316C90083121A
:101020005A088316C800CF01CE010330CD00E83046
:10103000CC008A118312FE238A157A088316CB000E
:101040007908CA007808C9007708C800CD01831262
:1010500062088316CC008A1183122A248A157A0822
:101060008316CF007908CE007808CD007708CC0031
:101070004D30D3005530D2000530D1008530D0003E
:101080008A11831249248A1577088316CC007808C0
:10109000CD007908CE007A08CF004B08D3004A086B
:1010A000D2004908D1004808D0008A118312C02418
:1010B0008A1583107A088316D3007908D20078083D
:1010C000D1007708D0004F08D7004E08D6004D0851
:1010D000D5004C08D4008A118312DD248A157A08C1
:1010E0008316D3007908D2007808D1007708D000A1
:1010F0008A11831223268A157A08E7007908E60008
:101100007808E5007708E400FD013B30FC00413041
:10111000840067088316CB00831266088316CA0012
:10112000831265088316C900831264088316C800F9
:101130008A11831288268A150D300317BA008A1186
:101140000313FC218A150A300317BA008A1103130E
:10115000FC218A158316C9013B30C8008A1183120D
:101160001D278A158A150A121F2BFD013B30FC0032
:10117000413084006B088316CB0083126A08831603
:10118000CA00831269088316C9008312680883168F
:10119000C8008A11831288268A150D300317BA00F9
:1011A0008A110313FC218A150A300317BA008A1129
:1011B0000313FC218A158316C9013B30C8008A112C
:1011C00083121D278A158A150A12532B8316480885
:1011D0000319AC29D4004C080319AC29D402031C10
:1011E000F6287F30D4070318AC29FC288130D402BC
:1011F000031CAC290319AC295408F700F801F901C4
:10120000FA01D3014908D200D2174A08D1004B088D
:10121000D0001930D4004F08D00203181F29013024
:10122000D10203181F29D20203181F29D302031861
:101230001F29D30AD20AD10A4F08D00751294E08D4
:10124000D10203183A290130D20203183A29D302F5
:1012500003183A29D30AD20A4E08D1074F08D007FB
:10126000031C5129D10A031D5129D20A031D5129FA
:10127000D30A51294D088038D20203185029013071
:10128000D30203185029D30A4D088038D2074E08DC
:10129000D107031C2E29D20A031D2E29D30A2E2979
:1012A0007A14D40B54295F290310D00DD10DD20D1F
:1012B000D30D0310FA0DF90DF80DD50D0B29551CA2
:1012C00067290310F80CF90CFA0CD50C6A29F703FE
:1012D0000319AC29D51B93290310D00DD10DD20DC4
:1012E000D30D4F08D00203187F290130D102031813
:1012F0007F29D20203187F29D302031CA2294E089A
:10130000D10203188A290130D20203188A29D30294
:10131000031CA2294D088038D202031893290130FA
:10132000D302031CA229FA0A031DA229F90A031DEC
:10133000A229F80A031DA229F70A0319AC29F80CFF
:10134000F90CFA0C4908D4004D08D406D41FAA2978
:10135000F817B029F813B029F701F801F901FA01DB
:1013600083128A150A12C62B83164908D0004D082D
:10137000D006D01FC02903110310C91B0314F32981
:101380004908D0004C08D1004808D1020319CE29E1
:10139000D01FF3290308013A8300F3294D08D10037
:1013A0004908D1020319DA29D01FF3290308013AA9
:1013B0008300F3294E08D1004A08D1020319E62917
:1013C000D01FF3290308013A8300F3294F08D10005
:1013D0004B08D1020319F229D01FF3290308013A5F
:1013E0008300F329031083128A150A12F82B83163F
:1013F0008C1083125708E1005608E0005508DF0002
:101400005408DE005908623CE30083168C148312F2
:101410008A150A12FD2B840183131F3083051930AE
:1014200083169900A6309800903083129800831696
:101430001F149F141F159F1107309C008312A901D0
:10144000AA014630AF00B0015130B100B2015330B3
:10145000B300B4015630B500B6014130B700B80151
:101460005230B900BA010330CF00D001D101D2010E
:10147000D301D401D501D601D701D801D901DA01B0
:10148000DB01DC01DD01DE01DF01E001E101E20160
:10149000E301E401E501E601E701E801E901EA0110
:1014A000EB016C10EC106C11EC116C12EC126C1363
:1014B000EC13ED01EE01F201FF30F300F401F50051
:1014C000FC01FD01F601FE018316BE01BF014310C0
:1014D00001130F308312D8006230D9000C30F700AE
:1014E000073081018130840083130008F039073808
:1014F000800064000008F739F719F039770480009C
:10150000853090004830F80005389200FF3083168F
:1015100092008A118312B9298A150B1683160C14AE
:101520008C148312071675127508831687008312B0
:101530008712F512750883168700831286108316AA
:101540008610831206118316061183120612831663
:1015500006121F1383121F179F1783169F138312E0
:101560001F1483161F109F141F159F150030F800BD
:1015700083121F08C73978049F0003081839F70041
:1015800083160E08033977040E148E148315031680
:101590000B3A83120319D02A133A0319F12AF22ABB
:1015A000FD013B30FC008316C80148088A118312F4
:1015B00056208A158316C80AF70083120317BA004B
:1015C0008A110313FC218A15053083164802031D76
:1015D000D52AC9013B30C8008A11831205238A1518
:1015E000F22AF22A64006D088316C800C9018A1124
:1015F0008312662B8A15F8080319862B8316C901F6
:101600007030C800CB012F30CA008A1183128D239D
:101610008A15F808031D102B8A11D42B8A15862BE6
:101620008316C9017030C800CB013130CA008A115D
:1016300083128D238A15F808031D202B0028862B82
:101640008316C9017030C800CB013330CA008A113B
:1016500083128D238A15F808031D322B8A11812FDE
:101660008A15862B8316C9017030C800CB0135302E
:10167000CA008A1183128D238A15F808031D442B92
:101680008A11C92F8A15862B8316C9017030C800AC
:10169000CB013730CA008A1183128D238A15F808CE
:1016A000031D542BB528862B8316C9017030C80042
:1016B000CB013930CA008A1183128D238A15F808AC
:1016C000031D662B8A11F12F8A15862BFD013B30F5
:1016D000FC008316C80148088A11831260208A150D
:1016E0008316C80AF70083120317BA008A1103137E
:1016F000FC218A150F3083164802031D6B2BC9018C
:101700003B30C8008A11831205238A156C1C9D2B5F
:10171000EC189D2B6C1A9D2B8A1188218A15DD08E7
:10172000031D9C2BDC08031D9C2BDB08031D9C2B3D
:101730005A083B3C03189D2B6C166C1C7F2CEC1933
:101740007F2C6C1A7F2C1F151F19A42B1E088316C3
:10175000CD01CC008A1183122A248A157A088316B7
:10176000C7007908C6007808C5007708C400470894
:10177000CB004608CA004508C9004408C800CF018C
:10178000CE01CD018730CC008312E628770883167E
:10179000C8007808C9007908CA007A08CB00CF00D1
:1017A0004A08CE004908CD004808CC00D301D20138
:1017B0002030D1008130D0008A11831249248A154B
:1017C0007A088316C7007908C6007808C50077082C
:1017D000C400CB01CA01C9018030C8004708CF004E
:1017E0004608CE004508CD004408CC008312B42939
:1017F0000318FC2B031D7F2CF72961088316CB00EF
:10180000831260088316CA0083125F088316C9001A
:1018100083125E088316C800CF01CE010330CD00CD
:10182000E830CC008A118312FE238A157A088316C9
:10183000CB007908CA007808C9007708C800CD0134
:10184000831263088316CC008A1183122A248A1516
:101850007A088316CF007908CE007808CD00770883
:10186000CC009630D3004330D2002330D1008230F8
:10187000D0008A11831249248A1577088316CC0078
:101880007808CD007908CE007A08CF004B08D30045
:101890004A08D2004908D1004808D0008A118312B2
:1018A000C0248A1583107A088316D3007908D200E1
:1018B0007808D1007708D0004F08D7004E08D6002E
:1018C0004D08D5004C08D4008A118312DD248A15F6
:1018D0007A088316D3007908D2007808D1007708F7
:1018E000D0008A11831223268A157A08EB00790822
:1018F000EA007808E9007708E800EC15EC176C1CA2
:0E190000852CEC18852C6C1E852CF22A6300B9
:02400E00753FFC
:00000001FF
